:030000000219FDE5
:03000B000200AA46
:03002B000201557A
:03005B000202E4BA
:030073000202D1B5
:1000800002030406080C10182030406080040608A3
:100090000C10182030406080A0C00003070F1F0D17
:1000A0000D0403060D0503030202C2AFC0D0C0E079
:1000B000206214E5256009E473E525F4F58AD2622F
:1000C000D0E0D0D0D2AF3285268AC262E526F46075
:1000D0003130682720720CE57BF45290D0E0D0D00C
:1000E000D2AF32E57BF45290206F1020660DE57B95
:1000F000F4D33333335290E57B4290D0E0D0D0D26A
:10010000AF32758A00C28DD26201FB01B930680737
:10011000206604D295D29201B9306807206604D2D5
:1001200094D29101B9306807206604D293D290012D
:10013000B9306807206604D295D29201B9306807B9
:10014000206604D294D29101B9306807206604D2A7
:1001500093D29001B9C2AFC2AD53E6EFC0D0C0E0B8
:10016000D2D3D2AFC2CEE52A6007207449152A2126
:10017000B67800790020742EE580307E01F430E7F7
:100180000278FF53DACF207E0343DA20307E034328
:10019000DA10C2D8C271E580307E01F430E702790E
:1001A000FFC3E89970CB306103752A402074037552
:1001B0002A40885CD27020740DE52B6004152B2139
:1001C000C643DA01C2D820700221D9A85C2061029E
:1001D000C27020740221D788227882B60403852257
:1001E00024C3E52594404002D26420CF0AD0E0D059
:1001F000D043E610D2AD32C2CF053A7802E52A608C
:1002000005307402152AC3E55C94014005755F0052
:100210004123756000756900E55F2401F55F5003B7
:10022000755FFF7982B7020D306E1DC3E5229432EF
:100230004016854C227982B7030E306E0BC3E5223F
:1002400094324004798E8722C3E5239522600840CA
:1002500004152341570523D8CA0569E569700215BD
:1002600069D56A63756A017805C3E569956B40577E
:10027000C3E569956C50087801756A0302028BC367
:10028000E569956D50057801756A01C3E5629524AD
:10029000401E7982B7040241BC206E14852462E5B9
:1002A00069046003856B69756A0175233C0202C7A6
:1002B000E5622850057562FF41BCF562E562047095
:1002C000067560FF7569FFD0E0D0D043E610D2AD6F
:1002D00032C2AF53E67F7592FA7593FFC260759193
:1002E00004D2AF32C2AF53E6EFC2ADC0D0C0E0C05F
:1002F000F0D2D3D2AFA8FBA9FCC2D8307102614BB7
:1003000053DACF207E0343DA10307E0343DA20D263
:1003100071E580307E01F420E70261228827892878
:10032000A13053DACF207E0343DA20307E0343DA54
:1003300010C2D8C271307402A11C7800E580307EF2
:1003400001F430E702A11C885CA10453DACF207EBF
:100350000343DA20307E0343DA10C2712061028148
:100360002453DACF207E0343DA10307E0343DA20B1
:10037000C2D8D27188578958C3E89555F8E995567F
:10038000F97B007E087A00C3E8948CE9940050055C
:10039000755B008116882178A2E6A8216055C3E824
:1003A00094C8E994005008E4D2E4FB7A0A61F1C3EE
:1003B000E89468E994015008E4D2E3FB7A0F61F114
:1003C000C3E894D0E994025008E4D2E2FB7A1E61BB
:1003D000F1C3E894A0E994055008E4D2E1FB7A3C2B
:1003E00061F1C3E89498E994085008E4D2E0FB7AFC
:1003F000787E00C3E89559FCE9955AFD30E70AEC90
:10040000F42401FCEDF43400FD755B00C3EC9AEDBF
:100410009E5003755B018859895A855755855856F2
:100420007802A104C3E89527F8E99528F9307C0201
:1004300081E8307B0281E8307A0281E12075028117
:1004400047E9FDE8FC8166E9C313F9E813F8307960
:100450000281E1E9C313F9E813F830780281E1E998
:10046000C313FDE813FC20612CC3EC941CED940233
:0F0470004002817DED701EC3EC94C85018052921
:10047F00E52970021529C3E529940A5002A11C75BC
:10048F005C00D270A11CE529600215297400207F41
:10049F00037896E624FAFEE43400FFC3EC9EFCEDED
:1004AF009FFD50067800790081E8C3EC94FFED942E
:1004BF0000400678FF790081E8EC8572F0A4C5F062
:1004CF00A2F733F87900400302050478FF790002A0
:1004DF000504E9C313F9E813F8307C0EE9600278DC
:1004EF00FFC3E81338F8E43400F9C3E894FFE99444
:1004FF0000400278FF885CD270206102A11C741F3B
:10050F00F4552F4BF52FC274EB7002D274752A403D
:10051F00307403752A0A306102A13020740353DA54
:10052F00FE207403752B20D0F0D0E0D0D0D2AD4395
:10053F00E6103279010205607903020560790A023B
:10054F000560791E020560796402056079C80205AD
:10055F00607817E4D5E0FDD8FAD9F6227A147B78C3
:10056F000205877A107B8C0205877A0D7BB4020512
:10057F00877A0B7BC80205877902E4C291D5E0FD2B
:10058F00D294D291D5E0FDC291D5E0FDC294D29123
:10059F00D5E0FDE920E004D295D29230E004D29369
:1005AF00D290E573D5E0FDE920E002C29230E0027F
:1005BF00C2907496D5E0FDD9C1EAF8D5E0FDD8FB1D
:1005CF00DBB6C29122C37C007D0075F00005F0EA16
:1005DF0033FAEB33FB50F6EB13FBEA13FAC3E9FFE5
:1005EF00E8FEE89AF8E99BF95004EFF9EEF8B3EC5E
:1005FF0033FCED33FDD5F0DFEDF9ECF822E889F0AF
:10060F008A20D2D4F8A9F07B0030F70B7BFFF424BB
:10061F0001F8E9F43400F9E88520F0A4ADF0F8E929
:10062F008520F0A4AFF0FEED2EF974003FFA7C04A4
:10063F00C3EA13FAE913F9E813F8DCF48BF030F797
:10064F000AE8F42401F8E9F43400F9E889F0C2D497
:10065F00F8A9F0227882B60403020702C3E55C947E
:10066F0019401EE52D54067018206E3678057994C2
:10067F00E7146007780A1460027812C3E5419840C6
:10068F001F306E098564627569FF756A01852224C2
:10069F00E4F544F545F546F547F548C26E02070205
:1006AF00D26E7994E7147013E523F43333F913F80A
:1006BF00E9540104F9E854FE0206F6E71414701425
:1006CF00E523F4333333F913F8E9540304F9E85409
:1006DF00FC0206FEE523F433333333F913F8E95400
:1006EF00070404F9E854F8C39440F8E99400F98832
:1006FF0044894522C3E54113F9E54013F8C3E544A6
:10070F0098F8E54599F9500CC3E89480E994FF40B7
:10071F001602073AC3E8947FE99400500302073AA0
:10072F00787F790002073A788079FF8849894A22D1
:10073F00E5492546F8E54A3547F9854A20E430076B
:10074F0001F43548FA30E709C3EA94F0401502077F
:10075F0078C3EA940F500302077878FF79FF7A0F76
:10076F00020778780079007AF0C3E5249561500A82
:10077F00C374019524500B020796E54A20E70E0239
:10078F000796E54A30E706884689478A482278A5C2
:10079F00E6FAC3E54933F8E54A33F9D10CE930E716
:1007AF000BC3E89480E994FF4013E1D0C3E8947F32
:1007BF00E994005002E1D0787F7900E1D078807918
:1007CF00FFE820E715C3E52398F84009C3E8940133
:1007DF0040030207F778010207F7E8F42401252305
:1007EF00F840030207F778FF884B2278A6E6FAA8AD
:1007FF0047A94812060CE930E70CC3E89401E994C5
:10080F00FF401602082CC3E894FFE994005003023E
:10081F00082C78FF790002082C780179FFE920E78E
:10082F0015C3E54B98F84009C3E89401400302084B
:10083F00537801020853E8F42401254BF8400302D2
:10084F00085378FF88242278FFC26420693D206A0C
:10085F0012D264C3E541940A4009C3E52594405080
:0E086F0002C26479A1E76023E541601F74FFB7
:10087D008541F0848539F0306A0375F005A4F8C51B
:10088D00F0600278FFC3E895645002A86488632283
:10089D00C3E5409440E5419401E56350031401AE76
:1008AD00046002F563227883E6F520120F5D75E88A
:1008BD009012054275E890E5E820ECFBA8BDA9BEB5
:1008CD0012101D756E55756F00C3740013FD7455B0
:1008DD00606613FC74552CFC74003DFDECFAEDFBC9
:1008ED00C3E89AE99B4014E56E2455F56EE56F3427
:1008FD0000F56FEA2CFAEB3DFB80E5AE6EAF6FC3F2
:10090D00E56F13F9E56E13F8C3E913F9E813F87AF7
:10091D0003C3E913F9E813F8DAF7AA201A70097579
:10092D006E00756F000209451AEA6008EE28FEEFA9
:10093D0039FFDAF88E6E8F6F2275E890227883E694
:10094D00FFE5E820ECF7A8BDA9BE0570C3E57094DE
:10095D00084052757000E9FA79A0E76044EA700723
:10096D00E571601B020980C3E895716010E5715057
:10097D0006600C1402098C0460F902098CE571F50E
:10098D0071C39472401B7561C0C3940440137561AB
:10099D0080C39404400B756140C39404400375619A
:1009AD000075BB0E22EFC39401601F7455601BC30D
:1009BD00E894FFE994035012C3E8956EE9956F50E2
:1009CD0009E561600C15610209DEE561F46002055F
:1009DD0061A861C3E524985002A824C3E89562403C
:1009ED000AA862E562F4600385626188258826E5C0
:1009FD0070B4070375BB1022743279A787F0A4C5B4
:100A0D00F0A2F733F8C3E895614002A86188228807
:100A1D0024882588268864227540007541F022C2FD
:100A2D00AF75C820A8CCA9CDAA3A30CF010A75C898
:100A3D0024D2AFAB3BAC3C883B893CC3E89BF8E987
:100A4D009C206908F930670261384195AD3D8A3DBA
:100A5D00F9EA9DFA600478FF79FFAE3EAF3F8B3E19
:100A6D008C3FA83BA93CC3E89EF8E99FF9C3E5413B
:100A7D0013FBE54013FAE82AF540E93BF541500632
:100A8D007540FF7541FF41DFAA40AB41AC40AD4120
:100A9D007E047F02C3EB940440021E1FC3EB940837
:100AAD0040021E1FC3ED13FDEC13FCDEF7C3EA9CE1
:100ABD00FAEB9DFBEF6009C3E913F9E813F8DFF7D3
:100ACD00EA28FAEB39FB8A408B4150067BFF8B40BD
:100ADD008B41C3EB94025002D2673069047F0361EE
:100AED000A7892E6FFC3E537948240110FC3E537CC
:100AFD0094A040010FC3EF940640027F057E02E5EE
:100B0D0041C4540FF9E541C454F0F8E540C4540F05
:100B1D0028F8C3E89EFAE99400FB4009C3EA940261
:100B2D00EB940050047A02E4FB6184AA40AB41EBE4
:100B3D00C4FEEAC4540F4EFCC3EA9CFAEB9400FBCE
:100B4D00C3E813C313F8EA28FAEB3400FB8A408B91
:100B5D0041C3EB94024002C2677802EBC4FE7B00F6
:100B6D00EAC4540F4EFAC3EA98FA4005C3940250F2
:100B7D00027A027892E6FF30600261848551928597
:100B8D005293D26043E680C3E49AF8E49BF9306750
:100B9D00028110E8FAE9FBD3E913FDE813FC885153
:100BAD008952C3EF94036038EF20E00DE82CF8E98B
:100BBD003DF9ECFAEDFB020BD9E828F8E939F9C358
:100BCD00E82402F8E93400F97AFE7BFFC3EF9403C1
:100BDD00400E8A538B54884D894E8C4F8D508144D5
:100BED00885389548A4D8B4E8C4F8D5030691275B8
:100BFD0053F07554FF754FF07550FF7551F07552E8
:100C0D00FF8144E8FAD3E813FC8851C3EF940360E5
:100C1D0020EF20E007E82CF8ECFA8130E8282402D8
:100C2D00F87AFEC3EF940340088A53884D8C4F81A8
:100C3D004488538A4D8C4FE568C3335002646BF57D
:100C4D0068306002814E753402D26043E680E52D36
:100C5D0054066034A840A941C3E913F9E813F8C359
:0F0C6D00E913F9E813F8306904E92440F9C2AF3C
:100C7C0053E67F759100C3E498F594E499F5957566
:100C8C009104D26043E680D2AF22D26575430075E1
:100C9C002000306C03752040020CB5D26575430002
:100CAC00752040306C037520007801790120672095
:100CBC00E52D54066002C2657914E541C313700139
:100CCC0004F8C3941440027814306904781B791B1F
:100CDC00206010E543600C306903D53404D26DA15B
:100CEC005791560543E59B5440B52002A14130690C
:100CFC000908C3E89940011881DC20650A08C3E89B
:100D0C0099400281B581DCC265C2AF53E67F759113
:100D1C00003067127594007595FE759104D260438E
:100D2C00E680D2AF81B5AE40AF41C3E49EF594E40A
:100D3C009FF595A126C3E5339401500281B530652A
:100D4C000281B5D802A15581DCC26DC2AF53E67FDA
:100D5C00759100855394855495759104854D9285B4
:100D6C004E93D26043E680D2AFE52D540660082046
:100D7C006A020533020D93306D0D206C0A20650755
:100D8C001581158102164E227800306405306502FB
:100D9C007801E53775F007A4F9E5F028F5F0E9A23C
:100DAC00F013A2F113A2F213F537C3947850037524
:100DBC003778C3E53795384007D266E57BF4529017
:100DCC00306002A1CC854F92855093D26043E6806F
:100DDC0022207D1AC2AF754202C291C295D29230C6
:100DEC006204D293D290D2AF759F1102101AC2AF87
:100DFC00754202C291C293D290306204D295D292C3
:100E0C00D2AF759F1102101A30724B207D24C2AFE5
:100E1C0075420390013D757B02C290C29030620610
:100E2C00D294D291C136C294D291D2AF759F0102A5
:100E3C00101AC2AF75420390013D757B02C292C27B
:100E4C0092306206D294D291C15AC294D291D2AF4E
:100E5C00759F2102101A207D1CC2AF7542039001B0
:100E6C0019757B02C290306204D294D291D2AF75C4
:100E7C009F0102101AC2AF754203900119757B02D3
:100E8C00C292306204D294D291D2AF759F210210DB
:100E9C001A207D1AC2AF754204C292C293D290300E
:100EAC006204D294D291D2AF759F2102101AC2AFB4
:100EBC00754204C290C295D292306204D294D291FF
:100ECC00D2AF759F0102101A30724B207D24C2AF35
:100EDC00754205900131757B04C291C29130620656
:100EEC00D295D292C1F6C295D292D2AF759F110211
:100EFC00101AC2AF754205900149757B01C291C2AF
:100F0C0091306206D293D290E11AC293D290D2AFB2
:100F1C00759F1102101A207D1CC2AF7542059001FD
:100F2C000D757B04C291306204D295D292D2AF750A
:100F3C009F1102101AC2AF754205900125757B01F5
:100F4C00C2913062E8D293D290D2AF759F11021049
:100F5C001A207D1AC2AF754206C290C294D291304B
:100F6C006204D295D292D2AF759F0102101AC2AF11
:100F7C00754206C292C294D291306204D293D2903E
:100F8C00D2AF759F2102101A30724B207D24C2AF54
:100F9C00754201900149757B01C292C29230620682
:100FAC00D293D290E1B6C293D290D2AF759F210268
:100FBC00101AC2AF754201900131757B04C290C208
:100FCC0090306206D295D292E1DAC295D292D2AF2B
:100FDC00759F0102101A207D1CC2AF754201900151
:100FEC0025757B01C292306204D293D290D2AF7538
:100FFC009F2102101AC2AF75420190010D757B043E
:10100C00C290306204D295D292D2AF759F01C26663
:10101C002290010B757B00C292C291C290C292C207
:10102C0091C290C262227880760708760708760112
:10103C000876040876FF0876FF08760A0876020818
:10104C007601087601788C76010876000876B4086B
:10105C0076FF0876FF0876FF0876030876FF087699
:0E106C00010876FF0876250876D00876780809
:10107A0076C80876040876FF0876010876000876AE
:10108A007A08760A0876010876010876000876FF5B
:10109A00087600227887E6FFC272BF0302D272780E
:1010AA0088C27DE630E102D27DC27E7889E630E1EF
:1010BA0002D27EC3EF94026008758E01D2730210C9
:1010CA00D0758E00C273227880E6149000809378DF
:1010DA00A5F67881E6149000809378A6F67886E6DD
:1010EA001490008D9378A7F6789FE6F8700108C3EC
:1010FA00E8941140027811E82828F56B256B256BD6
:10110A0028F56C256B2828F56D7886E6F539C394A1
:10111A00025003753902789CE67538FFB4020375EC
:10112A0038A0B4030375388278A3E61490009A9322
:10113A00F566111D22227896E6FA7897E6FB7888FA
:10114A00E6B40305C3EB940EFB307F047A007BFF01
:10115A00C3EB9AFCC3948250027C827572000572BA
:10116A00EC8572F0A4C3E5F0947D40F222D27F317F
:10117A00401205517A007B007C10120547E55C2A73
:10118A00FA74003BFBDCF37C04C3EB13FBEA13FAAF
:10119A00DCF7FEC27F314022E5EF20E6037520002E
:1011AA000520903FFFE520146006901FFF146000A1
:1011BA009304600375EF1253D9BF7581C043FF8052
:1011CA0012054275EF0243B203E5B3240220E70D8C
:1011DA00F521E5E320E0068521B343E301111D75FE
:1011EA0080FF75A40075F19175D47F75900075A57F
:1011FA003F75F23F75D50075A60175E241111DE4F0
:10120A00F8F6D8FD75680111321216A97898867316
:10121A00753001C2AF12055B12056B12055112053A
:10122A00721205511205791205511217CB12055B7C
:10123A0012055B120556C2AF78FA79FA308707D9D8
:10124A00FBD8F7021C00119E11D1313F314078982A
:10125A008673111D75881075890275C824759104E5
:10126A0075D84075A82275B80275E690759B807589
:10127A009D0075D10E75BC5875BB0E75BA1175E80F
:10128A0080120542D2AF1208B375360053DACF2066
:10129A007E0343DA20307E0343DA1043DA01C2D8F0
:1012AA00C27112055BD2617B037A0CE55B70077A27
:1012BA000CDB03021240120551207003021240C2D5
:1012CA0070E55CC3940240E1E52F541F855E5DF52D
:1012DA005EB55DD5DAD5C26153DACF207E0343DA33
:1012EA0020307E0343DA10C2D8C27178A2E67008B1
:1012FA00D274E52F54E0F52FC275752900120556F0
:10130A00307409C3E529940A4002D2751205477858
:10131A00023074027800C3E55C9840F0C2AF12054F
:10132A006B12056B12056BD2AF12055B754C00127E
:10133A000547788CE6C39401500302140FE530C3C5
:10134A009401500302140F207435C3E55C94FF50D6
:10135A000302140FC2AF120580D2AF120556C3E5BD
:10136A005C940150EFC2AF12056B12054C12056B6B
:10137A00D2AF120556C3E55C94FF40E90218507FCC
:10138A0005D27F3140120556C2AFC27F3140AE5CF2
:10139A00C3E55C947FD2AF4076120542C2AF120514
:1013AA0080D2AFDFDC3177C3EE94057897F6120569
:1013BA005B1216EA1217D37F0AD27F314012055602
:1013CA00C2AFC27F3140AE5CC3E55C947FD2AF50FE
:1013DA00E6120542C2AF12056B12054C12056BD21A
:1013EA00AFDFD63177EE24037896F612055B121634
:1013FA00EA1218021205563140C3E55C94FF500206
:10140A006151021850C3E55C954C4003855C4C124F
:10141A00055678017988E7B403027805C3E55C9834
:10142A0040026139C2AF120580120580120580D2CE
:10143A00AF12055B753000E4F531F5320531E5315F
:10144A00F4703E0532789AE67819146012783214EC
:10145A00600D787D14600878FA146003753200C351
:0F146A00E53298401C111D1205421532753100F4
:1014790078998673C2AF120580D2AF7898867312B5
:10148900055612054CE52A70053074024140780171
:101499002074027806C3E55C9840A2120556E52A35
:1014A9007003021240C2AF111DE4F522F523F524A1
:1014B900F525F526F567D2AF7885E6C333F565E4FA
:1014C900F544F545F546F547F548F570F52CF52D44
:1014D900F53775700875BB10120542120946E5E823
:1014E90020ECFBA8BDA9BEE97001F8887112094A70
:1014F90075700875BB10119EC2AF7561FF120A05A0
:10150900852261852262852263D2AF752201752405
:1015190001752501752601856069756A017888E676
:10152900B40307C27D307602D27DD268D2697533A1
:1015390000120F5D120F94120A25120A2C120A25A5
:10154900120A2C120A25120CA7120663120D941204
:101559000DDD120A2C120C96306E03120703206758
:101569000312085630670312089D120D94120E14C7
:10157900120A2C120CA7306E0312073F120D941297
:101589000E9D120A2C120C96306E0312079D120D35
:1015990094120ED4120A2C120CA7306E031207FAF9
:1015A900120D94120F5D120A2C120946120C961292
:1015B9000D94120F9412094A120A2C30692C856471
:1015C90061856462856069756A0179187A0CC3E579
:1015D90033994009C269D26A8A350215F3C3E55CB9
:1015E9009401400302154F021656306A1D206C1AE9
:1015F900E535147006C26AD26BA14FF535C3E55CB7
:101609009401400302154F021656753600C3E55F73
:1016190094014009856462856069756A0178FA797F
:10162900A4E760027803C3E55F985021307404E5AC
:101639002A601A78F0306C058564617820C3E54129
:10164900985002A14F0536E55C6002C15975360014
:10165900C2AF111D7887E6FE7602119E7887EEF6F5
:10166900E4F522F523F524F525F526F565752C0015
:10167900752D00D2AF120556111D78A4E6600CC273
:1016890095D292C294D291C293D290307406E52A2F
:1016990070024140788DE6C3940140026116814190
:1016A900901A0D782012172CE520B4A50CA3121757
:1016B9002CE520B45A030216CA11321216EA021690
:1016C900E9901A0378807B0A12172CA308DBF9909A
:1016D9001A0F788C7B1912172CA308DBF9901A289A
:1016E90022C2AF12176B121745901A00740E121707
:1016F90031A37406121731A37415121731901A0306
:1017090078807B0A121730A308DBF9901A0F788CBE
:101719007B19121730A308DBF912177E12175C9098
:101729001A2822E493F622E6438F01538FFD75EFC1
:101739000275B7A575B7F1F0538FFE22438F0243A7
:101749008F0175EF0275B7A575B7F1901A0DF053B2
:101759008FFC22901A0D74A5F131901A0E745AF16A
:1017690031227A3079D07820901A40F12CE520F78F
:1017790009A3DAF7227A3079D0901A40E7F13109D2
:10178900A3DAF922AB74A875BB01027980BB020206
:101799007981BB03027982BB04027994BB05027982
:1017A90083BB06027986BB07027992BB0802798757
:1017B900BB0902799CBB0A027988BB0B027989E8CB
:1017C900F7227C0512055BDCFB22C2AF12056B1206
:1017D900057212057912058012054C12056B120566
:1017E9007212057912058012054C12056B120572E9
:1017F900120579120580D2AF22C2AF1205801205F7
:101809007912057212056B12054C120580120579C1
:1018190012057212056B12054C1205801205791218
:10182900057212056BD2AF22AE74AF75C2AF120545
:101839006B12056B12056B12054CDEF21205801254
:10184900054CDFF8D2AF221217D31217CB1217CBE0
:1018590075740175750175760011317C05AD5C12E1
:0F186900055BC3ED955C70F5C3E55C9401400A27
:10187800C3E55C94FF403702189312178D1216EADD
:101888001217D3C2AF75EF121217CBDCD10576C38E
:10189800E5769403500280C21217CB0575E57414DF
:1018A80090009F93F808C3E57598500280A9121715
:1018B800CB1217CB0574C3E574940C5002809512B3
:0D18C80010321216EAC2AF75EF121217CBE4
:0319FD000211A232
:101A00000E061507070104FFFF0A020101A55A018E
:101A100000B4FFFFFF03FF01FF25D078C804FF01DA
:091A200000FF0A010100FF00FFB4
:101A400023454D41585F4C746E675F32304123200F
:101A500023424C48454C492346333930232020202B
:101A60002020202020202020202020202020202076
:101C0000C2AFC2D353D9BF7581C043B20343FF8073
:101C1000752438752503B1C975EF0275E24043F1AB
:101C20008053A47F75D4FFD2877DFA780379E67C50
:101C300010752200752300901DD67B0675249875BB
:101C400025013087028142208708D8FBD9F9DCF7CB
:101C500081B4308708D8FBD9F9DCF781B4B189E4C5
:101C600093A3C39A6004DDC381B4DBDBB17B600264
:101C7000812B7B08E493FAA3B15CDBF87A30B15C8A
:101C8000752200752300B17BEAFCEBFDC3ED94FEE9
:101C9000400EB17B8A278B28ED30E0048A828B834B
:101CA000B17B7AC270D8C3ED94FE601350CEBD00F4
:101CB00025EC60097520007521FF0200008100A855
:101CC00027A9280809D804D90281D3B17FEA89AAB3
:101CD000F281C50D81A0C3ED94035049EDA2E092BD
:101CE000007AC5C3E5829400E583941C50902000DF
:101CF00010438F02438F0175B7A575B7F1F030001F
:101D00001FA827A9280809438F01538FFDD804D99C
:101D100002A12089AAE275B7A575B7F1F0A3A10DBC
:101D2000538FFC817C7AC1BD030CE493A3FAB140CC
:101D3000DCF8B138817C817EAA22AB23B15CEBFA5E
:101D4000EA6222752608C3E52313F523E52213F57D
:101D50002250066323A0632201D526EAB1C9B1C986
:101D600075260AEAF4200102D287300102C287B147
:101D7000C9C3134002C201D526EB22B17FEAFB2082
:101D80008702A17F308702A184752608AE24AF2583
:101D9000C3EF13FFEE13FEB1CDB1C9C3EA13308711
:101DA000024480FA30E703632201C3E52313F523DD
:101DB000E52213F52250066323A0632201D526D91C
:101DC000E52265236523F52222AE24AF250E0FDE22
:101DD000FEDFFCD20122424C48656C693437316326
:041DE000F390060175
:00000001FF
